:030000000210FDEE
:03000B000200A54B
:03002B000202AB23
:03005B0002045C40
:030073000204364E
:1000800002030406080C10182030406080040608A3
:100090000C10182030406080A0C00D0D0403060D28
:1000A0000502030202C2AFC0D0C0E020620C20688B
:1000B00002419A306602415AE47385258AC262E59C
:1000C00025F470022121206802210E758B00D0E0FA
:1000D000D0D0D290D291D292D2AF32D290D291D20D
:1000E000927406D5E0FDE53C1420E21520E10D20D8
:1000F0007D02D295307D02D29302011ED29402017C
:100100001E207D02D293307D02D29502011E758B96
:1001100000D0E0D0D0D290D291D292D2AF32758BB3
:1001200000D0E0D0D0D2AF32419AE525600A207DE0
:1001300002C290307D02C292D291419AE5256002BE
:10014000C291207D02D292307D02D290419AE52563
:10015000600A207D02C292307D02C290207D02D2D0
:1001600090307D02D292419A207D02C293307D026E
:10017000C295207D02C295307D02C2937438D5E0CD
:10018000FDE525600A207D02C290307D02C292D238
:1001900091419A207D02C293307D02C295C294742F
:1001A00038D5E0FDE525600A207D02C290307D0251
:1001B000C292D291419AC294207D02C293307D02B4
:1001C000C2957438D5E0FDE5256002C291207D021C
:1001D000D292307D02D290419AC294207D02C29583
:1001E000307D02C2937438D5E0FDE5256002C291EE
:1001F000207D02D292307D02D290419A207D02C2AF
:1002000095307D02C293C2947438D5E0FDE5256037
:100210000A207D02C292307D02C290207D02D290DF
:10022000307D02D292419A207D02C295307D02C279
:1002300093207D02C293307D02C2957438D5E0FDD3
:10024000E525600A207D02C292307D02C290207DA9
:1002500002D290307D02D292419A30723DE53C202C
:10026000E21A20E129207D02C293307D02C295204E
:100270007D02C295307D02C29302029A20E1E620FF
:100280007D02C293307D02C295C29402029AC2944A
:10029000207D02C295307D02C293E525F4F58A7572
:1002A0008B00D262D0E0D0D0D2AF32C2AFC2AD5359
:1002B000E6EFC0D0C0E0D2D3D2AFC2CEE52960070E
:1002C0002074461529610978007900E580307E01A7
:1002D000F430E70278FF53DACF207E0343DA203090
:1002E0007E0343DA10C2D8C271E580307E01F4305B
:1002F000E70279FFC3E89970CE3061037529402089
:1003000074037529408859D270E52A6004152A6162
:100310001920740543DA01C2D82070026141A8593E
:10032000206102C270207402612A882230690AC3E7
:10033000E522955E4003855E227882B6040385221D
:1003400024C3E52594404002D26420CF0CD0E0D0F5
:10035000D0C2D343E610D2AD32C2CF7802E52960D5
:10036000053074021529C3E55994014005755C00F8
:100370006183755D00756400E55C2401F55C5003E4
:10038000755CFF7982B7020EE547601EC3E52294D3
:100390003240178546227982B7030FE547600BC3C9
:1003A000E52294324004798E8722C3E523952260AA
:1003B000084004152361B90523D8C80564E56470B5
:1003C000021564D565647565017805C3E5649566B5
:1003D0004058C3E5649567500878017565030203CA
:1003E000EDC3E564956850057801756501C3E55F67
:1003F0009524401F7982B70402811FE54770148558
:10040000245FE56404600385666475650175233CBB
:1004100002042AE55F285005755FFF811FF55FE53F
:100420005F047006755DFF7564FFD0E0D0D0C2D365
:1004300043E610D2AD32C0D0C0E0C2AF53917F537B
:10044000E67FC260759100C3E49550F594E4955140
:10045000F595759104D0E0D0D0D2AF32C2AF53E65B
:10046000EFC2ADC0D0C0E0C0F0D2D3D2AFA8FBA9DC
:0E047000FCC2D830710281C353DACF207E0364
:10047E0043DA10307E0343DA20D271E580307E01FC
:10048E00F420E702819A88268927C19A53DACF2071
:10049E007E0343DA20307E0343DA10C2D8C27130B5
:1004AE007402C1867800E580307E01F430E702C127
:1004BE00868859C16D53DACF207E0343DA20307E11
:1004CE000343DA10C271206102A19353DACF207E6A
:1004DE000343DA10307E0343DA20C2D8D271885437
:1004EE008955C3E89552F8E99553F9E4FB7E027AF3
:1004FE0000C3E8948CE994005005755800A183C39D
:10050E00E894C8E994005008E4D2E4FB7A0AA160AA
:10051E00C3E89468E994015008E4D2E3FB7A0FA192
:10052E0060C3E894D0E994025008E4D2E2FB7A1E4C
:10053E00A160C3E894A0E994055008E4D2E1FB7AE7
:10054E003CA160C3E89498E994085008E4D2E0FB1B
:10055E007A787E00C3E89556FCE99557FD30E7089A
:10056E00ECF42401FCEDF4FD755800C3EC9AED9EFD
:10057E00500375580188568957A854A95588528931
:10058E00537802C16DC3E89526F8E99527F9307CBA
:10059E0002C151307B02C151307A02C14A2075022C
:1005AE00A1B6E9FDE8FCA1D5E9C313F9E813F830CB
:1005BE007902C14AE9C313F9E813F8307802C14A47
:1005CE00E9C313FDE813FC206126C3EC941CED94E3
:1005DE00024002A1ECED7018C3EC94C8501205282D
:1005EE00C3E528940A5002C186755900D270C1869F
:1005FE00E528600215287400207F037896E624FA19
:10060E00FEE43400FFC3EC9EFCED9FFD5006780027
:10061E007900C151C3EC94FFED9400400678FF7948
:10062E0000C151EC856FF0A4C5F0A2F733F8790044
:10063E00400302066D78FF790002066DE9C313F9D7
:10064E00E813F8307C0EE9600278FFC3E81338F83F
:10065E00E43400F9C3E894FFE99400400278FF887F
:10066E0059D270206102C186741FF4552F4BF52F9D
:10067E00C274E42B7002D27475294030740375294C
:10068E000A306102C19A20740353DAFE752A2030B3
:10069E007403752A0AD0F0D0E0D0D0C2D3D2AD43C5
:1006AE00E6103279010206CF79030206CF790A02EB
:1006BE0006CF791E0206CF79640206CF79C80206EC
:1006CE00CF7817E4D5E0FDD8FAD9F6227A147B78E4
:1006DE000206F67A107B8C0206F67A0D7BB40206C1
:1006EE00F67A0B7BC80206F6AC257525017902B2A7
:1006FE007DE4C294D5E0FDE5256002C291D5E0FD12
:10070E00D291D5E0FDD294D5E0FDE525600A207D9D
:10071E0002C290307D02C292E570D5E0FD207D02CE
:10072E00D290307D02D2927496D5E0FDD9C1EAF80E
:10073E00D5E0FDD8FBDBB1C2948C2522C37C007DB5
:10074E000075F00005F0EA33FAEB33FB50F6EB13CD
:10075E00FBEA13FAC3E9FFE8FEE89AF8E99BF950C1
:10076E0004EFF9EEF8B3EC33FCED33FDD5F0DFED2D
:10077E00F9ECF822E889F08A20D2D4F8A9F07B00AF
:10078E0030F70B7BFFF42401F8E9F43400F9E88527
:10079E0020F0A4ADF0F8E98520F0A4AFF0FEED2E28
:1007AE00F974003FFA7C04C3EA13FAE913F9E8136B
:1007BE00F8DCF48BF030F70AE8F42401F8E9F434AD
:1007CE0000F9E889F0C2D4F8A9F0227882B60403C1
:1007DE0002087BC3E5599419401FE52D5406701984
:1007EE00E547703878057994E7146007780A146045
:1007FE00027812C3E53B984020E547600985615FAA
:10080E007564FF756501852224E4F53EF53FF540DC
:10081E00F541F542F54702087B7547017994E714D7
:10082E007013E523F43333F913F8E9540104F9E8AE
:10083E0054FE02086FE714147014E523F4333333B7
:10084E00F913F8E9540304F9E854FC020877E52398
:10085E00F433333333F913F8E954070404F9E85445
:0E086E00F8C39440F8E99400F9883E893F22CF
:10087C00E547603BC3E53B13F9E53A13F8C3E53EA6
:10088C0098F8E53F99F9500CC3E89480E994FF403F
:10089C00160208B7C3E8947FE9940050030208B726
:1008AC00787F79000208B7788079FF8843894422E1
:1008BC00E5476058E5432540F8E5443541F9854462
:1008CC0020E4300701F43542FA30E709C3EA94F02A
:1008DC0040150208F9C3EA940F50030208F978FF97
:1008EC0079FF7A0F0208F9780079007AF0C3E524D1
:1008FC00955E5006E52460092112E54420E70D21A0
:10090C0012E54430E706884089418A4222E5477067
:10091C000302097D78A1E6FAC3E54333F8E54433D5
:10092C00F9120782E930E70BC3E89480E994FF40A1
:10093C00132154C3E8947FE9940050022154787F2A
:10094C0079002154788079FFE820E715C3E52398D6
:10095C00F84009C3E89401400302097B78010209BD
:10096C007BE8F424012523F8400302097B78FF88F7
:10097C004522E54770030209E078A2E6FAA841A9EE
:10098C0042120782E930E70CC3E89401E994FF4076
:10099C00160209B7C3E894FFE9940050030209B7A3
:1009AC0078FF79000209B7780179FFE920E715C3D0
:1009BC00E54598F84009C3E8940140030209DE7844
:1009CC00000209DEE8F424012545F840030209DEA3
:1009DC0078FF88242278FFC264E52D5406702FD24C
:1009EC0064C3E53B940A4009C3E52594405002C218
:1009FC0064E53B601974FF853BF0848537F0A4F8FF
:100A0C00C5F0600278FFC3E895615002A861886068
:100A1C00227883E6F520120F1E75E8901206B17548
:100A2C00E890E5E820ECFBA8BDA9BE120F9E756B03
:100A3C0030756C00C3740013FD743013FC74302CCF
:100A4C00FC74003DFDECFAEDFBC3E89AE99B401405
:100A5C00E56B2430F56BE56C3400F56CEA2CFAEBA5
:100A6C003DFB80E5AE6BAF6CC3E56C13F9E56B1326
:100A7C00F8C3E913F9E813F8E56B28F569E56C3967
:100A8C00F56A7A03C3E913F9E813F8DAF7AA201A1E
:100A9C007009756B00756C00020AB71AEA6008EEF3
:100AAC0028FEEF39FFDAF88E6B8F6C2275E89022F6
:100ABC007883E6FFE5E820ECF7A8BDA9BE056DC379
:100ACC00E56D94084052756D00E9FA79A0E7604431
:100ADC00EA7007E56E601B020AF2C3E8956E6010BF
:100AEC00E56E5006600C14020AFE0460F9020AFE60
:100AFC00E56EF56EC3946D401B755EC0C3940440E7
:100B0C0013755E80C39404400B755E40C39404401F
:100B1C0003755E0075BB0622EFC39401601BC3E82E
:100B2C0094FFE994035012C3E8956BE9956C500956
:100B3C00E55E600C155E020B4CE55EF46002055E32
:100B4C00A85EC3E524985002A824C3E8955F400A28
:100B5C00A85FE55FF46003855F5E8825E56DB407EB
:100B6C000375BB1022743279A387F0A4C5F0A2F7E9
:100B7C0033F8C3E8955E4002A85E88228824882555
:100B8C00886122753A00753B7F2275C820A8CCA9D4
:100B9C00CD75C824AA38AB3988388939C3E89AF896
:100BAC00E99BF9AA3AAB3BAC3AAD3B7E047F02C35E
:100BBC00EB940440021E1FC3EB940840021E1FC39B
:100BCC00ED13FDEC13FCDEF7C3EA9CFAEB9DFBEF97
:100BDC006009C3E913F9E813F8DFF7EA28FAEB39EF
:100BEC00FB8A3A8B3B400122753AFF753BFF223062
:100BFC00600261FB854C50854D51D26043E68022EA
:100C0C007892E6FFC3E535948240010FC3E5359435
:100C1C00A040010FC3EF940640027F057E021E30F8
:100C2C0072010EC3E53B940350060E0E3072010E9A
:100C3C00C3E53B940250060E0E3072010EA93BA880
:100C4C003A7A04C3E913F9E813F8DAF7C3E89EF823
:100C5C00E99400F94009C3E89402E994005004783F
:0E0C6C0002E4F9E9FBE8FAC3E913FDE813FC22
:100C7A00884C894DC3EF94036037EF20E00DE82CD0
:100C8A00F8E93DF9ECFAEDFB020CA8E828F8E93995
:100C9A00F9C3E89402F8E99400F97A02E4FBC3EF95
:100CAA009403400D8A4E8B4F884889498C4A8D4B54
:100CBA0022884E894F8A488B498C4A8D4B22306054
:100CCA000281C8D26043E680E52D54066027A83A1F
:100CDA00A93BE53494085006E820E002A94D759135
:100CEA0000C3E498F594E499F595759104D260539C
:100CFA00917F43E68022D265753D00752000020D82
:100D0A0013D265753D00752040E52D54066002C278
:100D1A0065D2AF206005E53D60012278017A02C301
:100D2A00E53B940540027802C3E53B940A40027809
:100D3A0003C3E53B940F40027A03306904781E7AB4
:100D4A0001206007E53D6003D2AF22D2AF0000C2A6
:100D5A00AFC3E53BFB940F40027B0FEB04307301FA
:100D6A002320620123F93069027982E58BC3994015
:100D7A00D0053DEAFBE59BF45440B52004DBF6A11F
:100D8A00AF206502A113C265759100AE3AAF3BC3AD
:100D9A00E49EF594E49FF595759104D26053917F92
:100DAA0043E680A113306502A113D895D2AF223051
:100DBA00690B0534206016753400020DD720600DCA
:100DCA0020650A206B07158115810215B922A84EE4
:100DDA00A94F75910053917FC3E498F594E499F56E
:100DEA0095759104854850854951D26043E6802221
:100DFA0078003064053065027801E53575F007A49E
:100E0A00F9E5F028F5F0E9A2F013A2F113A2F21322
:100E1A00F535C394785003753578C3E53595364072
:100E2A0008D266D290D291D292306002C133854AFA
:100E3A0050854B51D26043E68022C2AFC293C2941E
:100E4A00C29530720B9001FC7438D5E0FD020E5A3F
:100E5A00207D02D293307D02D295759F11753C0296
:100E6A00020F99C2AF207D02D292307D02D2903019
:100E7A0072179001D9C294207D02C295307D02C2B8
:100E8A00937438D5E0FD020E9690013C306206E577
:100E9A00256002C291207D03759F21307D03759FD5
:100EAA0001753C03020F99C2AFC293C294C2953036
:100EBA00720B9001B67438D5E0FD020EC7207D0290
:100ECA00D295307D02D293207D03759F01307D0338
:100EDA00759F21753C04020F99C2AFD291307217E7
:100EEA00900193207D02C293307D02C295C2947410
:100EFA0038D5E0FD020F0490012A30620EE5256024
:100F0A000A207D02C290307D02C292759F11753C03
:100F1A0005020F99C2AFC293C294C29530720B9068
:100F2A0001687438D5E0FD020F34D294207D037530
:100F3A009F21307D03759F01753C06020F99C2AF50
:100F4A00207D02D290307D02D29230721F90022709
:100F5A00207D02C293307D02C295207D02C2953067
:100F6A007D02C2937438D5E0FD020F7990014E30AC
:100F7A00620EE525600A207D02C292307D02C2908F
:100F8A00207D03759F01307D03759F21753C01C249
:100F9A0066D2AF22900128D290D291D292C293C245
:100FAA0094C295C26222788076070876070876018D
:100FBA000876040876FF0876FF08760B087602089A
:100FCA007601087601788C76010876000876B408EE
:100FDA0076FF0876FF0876FF0876030876FF08761C
:100FEA00010876FF0876250876D00876780876C84C
:100FFA000876040876FF08760108760008767A08EB
:10100A007607087601227887E6FFC2727888C27D61
:10101A00E630E102D27DC27E7889E630E102D27EF4
:10102A00C3EF94026008758E01D27302103D758E6B
:10103A0000C273227880E6149000809378A1F67833
:10104A0081E6149000809378A2F6120F9E22788689
:10105A00E61490008D9378A3F6120F9E22789FE6ED
:0F106A00F8700108C3E8941140027811E82828B3
:10107900F5662566256628F56725662828F5682218
:10108900789CE67536FF75370CB402067536A0757F
:10109900370AB4030675368275370522227896E633
:1010A900FA7897E6FB307F047A007BFFC3EB9AFC62
:1010B900C3948250027C82756F00056FEC856FF0D6
:1010C900A4C3E5F0948040F222D27F11A61206C093
:1010D9007A007B007C101206B6E5592AFA74003BA7
:1010E900FBDCF37C04C3EB13FBEA13FADCF7FEC267
:1010F9007F11A622E5EF20E6037520000520903F29
:10110900FFE520146006901DFF146000930460033E
:1011190075EF12C2D353D9BF7581C043FF80120640
:10112900B175EF0243B203E5B3240420E702F5B336
:10113900120F9E7580FF75A40075F19175D47F75A6
:10114900900775A53F75F2FF75D50075A60175E283
:1011590041120FB01215F478988670C2AF1206CA00
:101169001206DA1206C01206E11206C01206E812C9
:1011790006C01217171206CA1206CA1206C5C2AF4E
:10118900E4F8F6D8FD78C879C8308707D9FBD8F7CD
:10119900021C00120FB01215F41110113E11581152
:1011A90067118911A511A678988670120F9E758806
:1011B9005075891275C82475910475D84075A8228F
:1011C90075B80275E690759B80759D0075D10E7591
:1011D900BC5875BB0675BA1175E8801206B1D2AF55
:1011E900120A1D43DA01C2D8C2711206CA7530014A
:1011F900D2617B037A0CE55870067A0CDB022187F1
:101209001206C02070022187C270E559C3940240BA
:10121900E3E52F541F855B5AF55BB55AD7DAD7C278
:101229006153DACF207E0343DA20307E0343DA109C
:10123900C2D8C271C2757528001206C5307409C3B7
:10124900E528940A4002D2751206B6780230740273
:101259007800C3E5599840F0C2AF1206DA1206DAEF
:101269001206DAD2AF1206CA7546001206B6788C93
:10127900E6C394015003021348E530C394015003B7
:10128900021348207435C3E55994FF5003021348EB
:10129900C2AF1206EFD2AF1206C5C3E55994015089
:1012A900EFC2AF1206DA1206BB1206DAD2AF120685
:1012B900C5C3E55994FF40E902179C7F05D27F1108
:1012C900A61206C5C2AFC27F11A6AE59C3E559948D
:1012D9007FD2AF40741206B1C2AF1206EFD2AFDFB0
:1012E900DC11D2C3EE94057897F61206CA121636A7
:1012F90012171F7F0AD27F11A61206C5C2AFC27F7D
:1013090011A6AE59C3E559947FD2AF50E61206B182
:10131900C2AF1206DA1206BB1206DAD2AFDFD61155
:10132900D2EE24057896F61206CA12163612174E10
:101339001206C511A6C3E55994FF40F402179CC3D0
:10134900E559954640038559461206C578017988BD
:10135900E7B403027805C3E5599840024174C2AF66
:101369001206EF1206EF1206EFD2AF1206CA753057
:1013790000E4F531F5320531E531F470390532789B
:101389009AE67819146012783214600D787D146029
:101399000878FA146003753200C3E53298401715CE
:1013A900327531B478998670C2AF1206EFD2AF7830
:1013B9009886701206C51206BBE5297005307402BD
:1013C900218778012074027806C3E5599840A7124D
:1013D90006C5E52970022187C2AF120F9EE4F522E6
:1013E900F523F524F525D2AF78858662F53EF53FDC
:1013F900F540F541F542F56DF547F52CF52DF53537
:10140900120B8F756D0875BB101206B1120AB8E57B
:10141900E820ECFBA8BDA9BEE97001F8886E120AA4
:10142900BC756D0875BB107887E6FE7602111078D9
:1014390087EEF6C2AF755EFF120B7185225E8522BB
:101449005F852260D2AF752201752401752501855A
:101459005D64756501D268D269753400120F1E1278
:0E1469000F48120B8F120B96120C0C021482FD
:10147700120F9E1110756D0075BB06120D0B120D24
:10148700B9120DD81207D9120DFA120E44120B9683
:10149700120BFB120C0C120CC8120D00120DB91214
:1014A7000DD812087C1209E1120DFA120E6D120BFB
:1014B70096120BFB120C0C120CC8120D0B120DB965
:1014C700120DD81208BC120DFA120EB1120B961299
:1014D7000BFB120C0C120CC8120D00120DB9120DD9
:1014E700D8120919120DFA120EE3120B96120BFB02
:1014F700120C0C120CC8120D0B120DB9120DD812CA
:10150700097E120DFA120F1E120B96120BFB120C0C
:101517000C120CC8120D00120AB8120DB9120DD810
:10152700120ABC120DFA120F48120B96120BFB127D
:101537000C0C120CC830692F206B2C85615E8561FD
:101547005F855D6475650179327A0AC3E534994030
:1015570009C269D26A8A3302156EC3E559940140FC
:10156700030214820215B9306A1B206B18E5331485
:101577007004C26A8177F533C3E5599401400302C9
:1015870014820215B9C3E55C9401400985615F8542
:101597005D64756501C3E55C94FA5016307404E523
:1015A70029600FC3E53B78F0306B027860985002F2
:1015B7008182C2AF120F9E7887E6FE7602111078FD
:1015C70087EEF6E4F522F523F524F525F562C268E2
:1015D700D2AF1206B1120F9E307406E529700221B0
:1015E70087788DE6C3940140024151617A901A0DC4
:1015F7007820121678E520B4A50CA3121678E520FA
:10160700B45A03021616120FB01216360216359088
:101617001A0378807B0A121678A308DBF9901A0F51
:10162700788C7B15121678A308DBF9901A2422C24E
:10163700AF1216B7121691901A00740D12167DA3E9
:10164700740212167DA3741312167D901A03788004
:101657007B0A12167CA308DBF9901A0F788C7B158E
:1016670012167CA308DBF91216CA1216A8901A24C0
:1016770022E493F622E6438F01538FFD75EF02753F
:10168700B7A575B7F1F0538FFE22438F02438F0141
:1016970075EF0275B7A575B7F1901A0DF0538FFC6A
:1016A70022901A0D74A5D17D901A0E745AD17D22FD
:1016B7007A3079D07820901A40D178E520F709A3BD
:1016C700DAF7227A3079D0901A40E7D17D09A3DA88
:1016D700F922AB71A872BB01027980BB0202798142
:1016E700BB03027982BB04027994BB05027983BBF1
:1016F70006027986BB07027992BB08027987BB0984
:1017070002799CBB0A027988BB0B027989E8F72228
:101717007C051206CADCFB22C2AF1206DA1206E10A
:101727001206E81206EF1206BB1206DA1206E112DB
:1017370006E81206EF1206BB1206DA1206E11206D7
:10174700E81206EFD2AF22C2AF1206EF1206E81276
:1017570006E11206DA1206BB1206EF1206E81206B7
:10176700E11206DA1206BB1206EF1206E81206E1CC
:101777001206DAD2AF22AE71AF72C2AF1206DA1218
:1017870006DA1206DA1206BBDEF21206EF1206BB03
:10179700DFF8D2AF22F11FF117F1177571017572DA
:1017A70001757300F17D7C05AD591206CAC3ED952D
:1017B7005970F5C3E5599401400AC3E55994FF40B0
:1017C700320217D8D1D9D136F11FC2AF75EF12F156
:1017D70017DCD50573C3E5739403500280C6F11770
:1017E7000572E5711490009A93F808C3E572985052
:1017F7000280AEF117F1170571C3E571940C500221
:10180700809C120FB0121636C2AF75EF121217175F
:101A00000D021307070104FFFF0B020101A55A0194
:101A100000B4FFFFFF03FF01FF25D078C804FF01DA
:051A200000FF0701FFBB
:101A400023506F6C61726973546472313241232088
:101A500023424C48454C4923463333302320202031
:101A60002020202020202020202020202020202076
:101C0000C2AFC2D353D9BF7581C043B20343FF8073
:101C1000752438752503B1BF75EF0275E24043F1B5
:101C20008053A47FD287780379E67C1075220075F3
:101C30002300901DCC7B0675249875250130870202
:101C4000813D208708D8FBD9F9DCF781AD308708C2
:101C5000D8FBD9F9DCF781ADB17FE493A3C39A60D7
:101C6000028126DBDDB171600281267B08E493FAF4
:101C7000A3B152DBF87A30B152752200752300B15E
:101C800071EAFCEBFDC3ED94FE400EB1718A278B27
:101C900028ED30E0048A828B83B1717AC270D8C398
:101CA000ED94FE601050CEBD0022EC600675200061
:101CB0000200008100A827A9280809D804D90281B8
:101CC000C9B175EA89AAF281BB0D8199C3ED94036C
:101CD0005049EDA2E092007AC5C3E5829400E58305
:101CE000941C5093200010438F02438F0175B7A5B9
:101CF00075B7F1F030001FA827A9280809438F0104
:101D0000538FFDD804D902A11689AAE275B7A5752B
:101D1000B7F1F0A3A103538FFC81757AC1BD030C09
:101D2000E493A3FAB136DCF8B12E81758177AA224B
:101D3000AB23B152EBFAEA6222752608C3E52313FE
:101D4000F523E52213F52250066323A0632201D573
:101D500026EAB1BFB1BF75260AEAF4200102D28794
:101D6000300102C287B1BFC3134002C201D526EBC6
:101D700022B175EAFB208702A175308702A17A752E
:101D80002608AE24AF25C3EF13FFEE13FEB1C3B197
:101D9000BFC3EA133087024480FA30E703632201AD
:101DA000C3E52313F523E52213F52250066323A090
:101DB000632201D526D9E52265236523F52222AECB
:101DC00024AF250E0FDEFEDFFCD20122424C486517
:0A1DD0006C6934373132F33006013C
:00000001FF
